:020000040000FA
:020000003A289C
:080008003A288C0081018316E7
:100010000313C030810508008C008101831603138F
:10002000C030810501308104831203130B110B1DB5
:1000300017288C0B162808008E00E13086050E0D5F
:100040001E398604080086132628861706138F009B
:100050000F080F0E1C2033200F081C203320E13026
:1000600086058613080001300C20861686120130A2
:100070000C20080083160313013086058312031336
:10008000861206138613E130860504300C200330F7
:100090001C20332001300C2008301C20332001307C
:1000A0000C2002301C20332001300C20283023206B
:1000B0000C3023200130232008300C204030232036
:1000C00006302520413023200830252042302320CF
:1000D00004302520433023200A30252044302320BB
:1000E0001130252045302320113025204630232093
:1000F0000E30252047302320003025204830232093
:100100000E30252049302320113025204A3023206D
:10011000113025204B302320113025204C30232056
:10012000113025204D3023200A3025204E30232049
:100130001B3025204F302320003025208030232005
:10014000433025206830252061302520723025205D
:10015000613025206330252074302520653025202E
:1001600072302520733025203A302520203025207C
:100170000030252001302520C0302320E03025200C
:10018000E1302520E2302520E3302520E430252011
:10019000E5302520E8302520EF302520F3302520DC
:1001A000F4302520F5302520F6302520F7302520A5
:1001B000F8302520FD30252014300520073013208D
:1001C0000130232050302520493025204330252080
:1001D0003130252036302520463025203830252066
:1001E00034302520203025204C3025204330252058
:1001F000443025207430252065302520733025209B
:100200007430252003309200C43023202A3025206A
:1002100080300C202A30252080300C202A302520E8
:1002200080300C202A30252080300C202A302520D8
:1002300080300C202A30252080300C202A302520C8
:1002400080300C202A30252080300C20C430232020
:10025000203025202030252020302520203025204A
:100260002030252020302520203025200430232058
:100270002A30252080300C202A30252080300C2088
:100280002A30252080300C202A30252080300C2078
:100290002A30252080300C202A30252080300C2068
:1002A0002A30252080300C202A30252080300C2058
:1002B000CB30232020302520203025202030252041
:1002C00020302520203025202030252020302520DA
:1002D00006302320920B04292030252008300520E9
:1002E0000730132001302320D43023204C30252028
:1002F000693025206E3025206530252020302520CE
:1003000034302520943023204C302520693025209E
:100310006E302520653025202030252033302520E3
:10032000C03023204C302520693025206E30252018
:1003300065302520203025203230252080302320B4
:100340004C302520693025206E3025206530252051
:100350002030252031302520103005200730132093
:100360000230232050309200FF302520920BB42918
:10037000103005200730132002302320FE302520C6
:100380000230920028309300A0300C201C30232033
:10039000930BC42902302320FF302520C0302320B6
:1003A000FE302520920BC22901302320FF300C2083
:1003B0008030232048302520653025206C302520D2
:1003C0006C3025206F30252020302520FF300C2078
:1003D000C13023202030252020302520203025202A
:1003E000573025206F302520723025206C30252095
:1003F0006430252007309200C0300C201C302320B0
:10040000920BFC29FF300C2080302320483025201F
:1004100065302520723025206530252027302520A5
:1004200073302520FF300C20C13023205030252090
:1004300049302520433025203130252036302520F5
:1004400046302520383025203430252007309200D2
:0E045000C0300C2018302320920B282AD62909
:02400E00F23F7F
:00000001FF
